Archive member included to satisfy reference by file (symbol)

/usr/local/mcuxpressoide-10.3.1_2233/ide/plugins/com.nxp.mcuxpresso.tools.linux_10.3.0.201811011841/tools/bin/../lib/gcc/arm-none-eabi/7.3.1/../../../../arm-none-eabi/lib/thumb/v7-m/libcr_c.a(__weak__main.o)
                              ./src/cr_startup_lpc175x_6x.o (__main)

Discarded input sections

 .group         0x0000000000000000        0xc ./src/PWM_GENUINO_CASI.o
 .group         0x0000000000000000        0xc ./src/PWM_GENUINO_CASI.o
 .group         0x0000000000000000        0xc ./src/PWM_GENUINO_CASI.o
 .group         0x0000000000000000        0xc ./src/PWM_GENUINO_CASI.o
 .group         0x0000000000000000        0xc ./src/PWM_GENUINO_CASI.o
 .group         0x0000000000000000        0xc ./src/PWM_GENUINO_CASI.o
 .group         0x0000000000000000        0xc ./src/PWM_GENUINO_CASI.o
 .text          0x0000000000000000        0x0 ./src/PWM_GENUINO_CASI.o
 .data          0x0000000000000000        0x0 ./src/PWM_GENUINO_CASI.o
 .bss           0x0000000000000000        0x0 ./src/PWM_GENUINO_CASI.o
 .group         0x0000000000000000        0xc ./src/Timer0.o
 .group         0x0000000000000000        0xc ./src/Timer0.o
 .group         0x0000000000000000        0xc ./src/Timer0.o
 .group         0x0000000000000000        0xc ./src/Timer0.o
 .group         0x0000000000000000        0xc ./src/Timer0.o
 .group         0x0000000000000000        0xc ./src/Timer0.o
 .text          0x0000000000000000        0x0 ./src/Timer0.o
 .data          0x0000000000000000        0x0 ./src/Timer0.o
Memory Configuration

Name             Origin             Length             Attributes
MFlash512        0x0000000000000000 0x0000000000080000 xr
RamLoc32         0x0000000010000000 0x0000000000008000 xrw
RamAHB32         0x000000002007c000 0x0000000000008000 xrw
*default*        0x0000000000000000 0xffffffffffffffff

Linker script and memory map

LOAD ./src/PWM_GENUINO_CASI.o
LOAD ./src/Timer0.o
LOAD ./src/cr_startup_lpc175x_6x.o
LOAD ./src/crp.o
LOAD ./src/gpio.o
LOAD ./src/mainPWM.o
START GROUP
LOAD /usr/local/mcuxpressoide-10.3.1_2233/ide/plugins/com.nxp.mcuxpresso.tools.linux_10.3.0.201811011841/tools/bin/../lib/gcc/arm-none-eabi/7.3.1/../../../../arm-none-eabi/lib/thumb/v7-m/libcr_c.a
LOAD /usr/local/mcuxpressoide-10.3.1_2233/ide/plugins/com.nxp.mcuxpresso.tools.linux_10.3.0.201811011841/tools/bin/../lib/gcc/arm-none-eabi/7.3.1/thumb/v7-m/libcr_eabihelpers.a
LOAD /usr/local/mcuxpressoide-10.3.1_2233/ide/plugins/com.nxp.mcuxpresso.tools.linux_10.3.0.201811011841/tools/bin/../lib/gcc/arm-none-eabi/7.3.1/thumb/v7-m/libgcc.a
END GROUP
                0x0000000000000000                __base_MFlash512 = 0x0
                0x0000000000000000                __base_Flash = 0x0
                0x0000000000080000                __top_MFlash512 = 0x80000
                0x0000000000080000                __top_Flash = 0x80000
                0x0000000010000000                __base_RamLoc32 = 0x10000000
                0x0000000010000000                __base_RAM = 0x10000000
                0x0000000010008000                __top_RamLoc32 = 0x10008000
                0x0000000010008000                __top_RAM = 0x10008000
                0x000000002007c000                __base_RamAHB32 = 0x2007c000
                0x000000002007c000                __base_RAM2 = 0x2007c000
                0x0000000020084000                __top_RamAHB32 = 0x20084000
                0x0000000020084000                __top_RAM2 = 0x20084000

.text           0x0000000000000000      0x888
 FILL mask 0xff
                0x0000000000000000                __vectors_start__ = ABSOLUTE (.)
 *(.isr_vector)
 .isr_vector    0x0000000000000000       0xcc ./src/cr_startup_lpc175x_6x.o
                0x0000000000000000                g_pfnVectors
                0x00000000000000cc                . = ALIGN (0x4)
                0x00000000000000cc                __section_table_start = .
                0x00000000000000cc                __data_section_table = .
                0x00000000000000cc        0x4 LONG 0x888 LOADADDR (.data)
                0x00000000000000d0        0x4 LONG 0x10000000 ADDR (.data)
                0x00000000000000d4        0x4 LONG 0xc SIZEOF (.data)
                0x00000000000000d8        0x4 LONG 0x888 LOADADDR (.data_RAM2)
                0x00000000000000dc        0x4 LONG 0x2007c000 ADDR (.data_RAM2)
                0x00000000000000e0        0x4 LONG 0x0 SIZEOF (.data_RAM2)
                0x00000000000000e4                __data_section_table_end = .
                0x00000000000000e4                __bss_section_table = .
                0x00000000000000e4        0x4 LONG 0x1000000c ADDR (.bss)
                0x00000000000000e8        0x4 LONG 0x10 SIZEOF (.bss)
                0x00000000000000ec        0x4 LONG 0x2007c000 ADDR (.bss_RAM2)
                0x00000000000000f0        0x4 LONG 0x0 SIZEOF (.bss_RAM2)
                0x00000000000000f4                __bss_section_table_end = .
                0x00000000000000f4                __section_table_end = .
 *(.after_vectors*)
 .after_vectors
                0x00000000000000f4      0x128 ./src/cr_startup_lpc175x_6x.o
                0x00000000000000f4                data_init
                0x0000000000000136                bss_init
                0x000000000000016c                ResetISR
                0x00000000000001e0                NMI_Handler
                0x00000000000001e6                HardFault_Handler
                0x00000000000001ec                MemManage_Handler
                0x00000000000001f2                BusFault_Handler
                0x00000000000001f8                UsageFault_Handler
                0x00000000000001fe                SVC_Handler
                0x0000000000000204                DebugMon_Handler
                0x000000000000020a                PendSV_Handler
                0x0000000000000210                SysTick_Handler
                0x0000000000000216                TIMER2_IRQHandler
                0x0000000000000216                RIT_IRQHandler
                0x0000000000000216                I2C0_IRQHandler
                0x0000000000000216                USBActivity_IRQHandler
                0x0000000000000216                PWM1_IRQHandler
                0x0000000000000216                I2C1_IRQHandler
                0x0000000000000216                EINT2_IRQHandler
                0x0000000000000216                UART1_IRQHandler
                0x0000000000000216                EINT3_IRQHandler
                0x0000000000000216                CANActivity_IRQHandler
                0x0000000000000216                TIMER3_IRQHandler
                0x0000000000000216                UART0_IRQHandler
                0x0000000000000216                IntDefaultHandler
                0x0000000000000216                PLL0_IRQHandler
                0x0000000000000216                CAN_IRQHandler
                0x0000000000000216                PLL1_IRQHandler
                0x0000000000000216                SSP0_IRQHandler
                0x0000000000000216                I2S_IRQHandler
                0x0000000000000216                I2C2_IRQHandler
                0x0000000000000216                RTC_IRQHandler
                0x0000000000000216                SPI_IRQHandler
                0x0000000000000216                EINT1_IRQHandler
                0x0000000000000216                TIMER1_IRQHandler
                0x0000000000000216                UART2_IRQHandler
                0x0000000000000216                ADC_IRQHandler
                0x0000000000000216                SSP1_IRQHandler
                0x0000000000000216                USB_IRQHandler
                0x0000000000000216                BOD_IRQHandler
                0x0000000000000216                WDT_IRQHandler
                0x0000000000000216                QEI_IRQHandler
                0x0000000000000216                EINT0_IRQHandler
                0x0000000000000216                DMA_IRQHandler
                0x0000000000000216                UART3_IRQHandler
                0x0000000000000216                MCPWM_IRQHandler
                0x0000000000000216                ENET_IRQHandler
                0x00000000000002fc                . = 0x2fc
 *fill*         0x000000000000021c       0xe0 ff
                0x00000000000002fc                PROVIDE (__CRP_WORD_START__ = .)
 *(.crp)
 .crp           0x00000000000002fc        0x4 ./src/crp.o
                0x00000000000002fc                CRP_WORD
                0x0000000000000300                PROVIDE (__CRP_WORD_END__ = .)
                0x0000000000000001                ASSERT (! ((__CRP_WORD_START__ == __CRP_WORD_END__)), Linker CRP Enabled, but no CRP_WORD provided within application)
 *(.text*)
 .text.initAll  0x0000000000000300       0x18 ./src/PWM_GENUINO_CASI.o
                0x0000000000000300                initAll
 .text.initPLL  0x0000000000000318      0x140 ./src/PWM_GENUINO_CASI.o
                0x0000000000000318                initPLL
 .text.initPinPWM
                0x0000000000000458       0x12 ./src/PWM_GENUINO_CASI.o
                0x0000000000000458                initPinPWM
 *fill*         0x000000000000046a        0x2 ff
 .text.initPWM  0x000000000000046c       0xbc ./src/PWM_GENUINO_CASI.o
                0x000000000000046c                initPWM
 .text.updateMR1
                0x0000000000000528      0x154 ./src/PWM_GENUINO_CASI.o
                0x0000000000000528                updateMR1
 .text.InitTimer0
                0x000000000000067c       0xc4 ./src/Timer0.o
                0x000000000000067c                InitTimer0
 .text.TIMER0_IRQHandler
                0x0000000000000740       0x30 ./src/Timer0.o
                0x0000000000000740                TIMER0_IRQHandler
 .text.SetPINSEL
                0x0000000000000770       0x8a ./src/gpio.o
                0x0000000000000770                SetPINSEL
 *fill*         0x00000000000007fa        0x2 ff
 .text.main     0x00000000000007fc       0x88 ./src/mainPWM.o
                0x00000000000007fc                main
 .text.__weak_main
                0x0000000000000884        0x4 /usr/local/mcuxpressoide-10.3.1_2233/ide/plugins/com.nxp.mcuxpresso.tools.linux_10.3.0.201811011841/tools/bin/../lib/gcc/arm-none-eabi/7.3.1/../../../../arm-none-eabi/lib/thumb/v7-m/libcr_c.a(__weak__main.o)
                0x0000000000000884                __main
                0x0000000000000884                __weak_main
 *(.rodata .rodata.* .constdata .constdata.*)
                0x0000000000000888                . = ALIGN (0x4)

.glue_7         0x0000000000000888        0x0
 .glue_7        0x0000000000000888        0x0 linker stubs

.glue_7t        0x0000000000000888        0x0
 .glue_7t       0x0000000000000888        0x0 linker stubs

.vfp11_veneer   0x0000000000000888        0x0
 .vfp11_veneer  0x0000000000000888        0x0 linker stubs

.v4_bx          0x0000000000000888        0x0
 .v4_bx         0x0000000000000888        0x0 linker stubs

.iplt           0x0000000000000888        0x0
 .iplt          0x0000000000000888        0x0 ./src/PWM_GENUINO_CASI.o

.rel.dyn        0x0000000000000888        0x0
 .rel.iplt      0x0000000000000888        0x0 ./src/PWM_GENUINO_CASI.o

.ARM.extab
 *(.ARM.extab* .gnu.linkonce.armextab.*)
                0x0000000000000888                __exidx_start = .

.ARM.exidx
 *(.ARM.exidx* .gnu.linkonce.armexidx.*)
                0x0000000000000888                __exidx_end = .
                0x0000000000000888                _etext = .

.data_RAM2      0x000000002007c000        0x0 load address 0x0000000000000888
 FILL mask 0xff
                [!provide]                        PROVIDE (__start_data_RAM2 = .)
 *(.ramfunc.$RAM2)
 *(.ramfunc.$RamAHB32)
 *(.data.$RAM2*)
 *(.data.$RamAHB32*)
                0x000000002007c000                . = ALIGN (0x4)
                [!provide]                        PROVIDE (__end_data_RAM2 = .)

.uninit_RESERVED
                0x0000000010000000        0x0
 *(.bss.$RESERVED*)
                0x0000000010000000                . = ALIGN (0x4)
                0x0000000010000000                _end_uninit_RESERVED = .

.data           0x0000000010000000        0xc load address 0x0000000000000888
 FILL mask 0xff
                0x0000000010000000                _data = .
 *(vtable)
 *(.ramfunc*)
 *(.data*)
 .data.movementLeft.3717
                0x0000000010000000        0x4 ./src/PWM_GENUINO_CASI.o
 .data.GradosActualizadosDelQT
                0x0000000010000004        0x4 ./src/mainPWM.o
                0x0000000010000004                GradosActualizadosDelQT
 .data.estadoServo.3689
                0x0000000010000008        0x4 ./src/mainPWM.o
                0x000000001000000c                . = ALIGN (0x4)
                0x000000001000000c                _edata = .

.igot.plt       0x000000001000000c        0x0 load address 0x0000000000000894
 .igot.plt      0x000000001000000c        0x0 ./src/PWM_GENUINO_CASI.o

.bss_RAM2       0x000000002007c000        0x0
                [!provide]                        PROVIDE (__start_bss_RAM2 = .)
 *(.bss.$RAM2*)
 *(.bss.$RamAHB32*)
                0x000000002007c000                . = ALIGN ((. != 0x0)?0x4:0x1)
                [!provide]                        PROVIDE (__end_bss_RAM2 = .)

.bss            0x000000001000000c       0x10
                0x000000001000000c                _bss = .
 *(.bss*)
 .bss.actualPlace
                0x000000001000000c        0x4 ./src/PWM_GENUINO_CASI.o
 .bss.direction.3718
                0x0000000010000010        0x4 ./src/PWM_GENUINO_CASI.o
 .bss.flagT0    0x0000000010000014        0x4 ./src/mainPWM.o
                0x0000000010000014                flagT0
 .bss.flagCambioAlgoElQT
                0x0000000010000018        0x4 ./src/mainPWM.o
                0x0000000010000018                flagCambioAlgoElQT
 *(COMMON)
                0x000000001000001c                . = ALIGN (0x4)
                0x000000001000001c                _ebss = .
                [!provide]                        PROVIDE (end = .)

.noinit_RAM2    0x000000002007c000        0x0
 *(.noinit.$RAM2*)
 *(.noinit.$RamAHB32*)
                0x000000002007c000                . = ALIGN (0x4)

.noinit         0x000000001000001c        0x0
                0x000000001000001c                _noinit = .
 *(.noinit*)
                0x000000001000001c                . = ALIGN (0x4)
                0x000000001000001c                _end_noinit = .
                [!provide]                        PROVIDE (_pvHeapStart = DEFINED (__user_heap_base)?__user_heap_base:.)
                0x0000000010008000                PROVIDE (_vStackTop = DEFINED (__user_stack_top)?__user_stack_top:(__top_RamLoc32 - 0x0))
                0xffffffffefff74f2                PROVIDE (__valid_user_code_checksum = (0x0 - ((((((_vStackTop + (ResetISR + 0x1)) + (NMI_Handler + 0x1)) + (HardFault_Handler + 0x1)) + (DEFINED (MemManage_Handler)?MemManage_Handler:0x0 + 0x1)) + (DEFINED (BusFault_Handler)?BusFault_Handler:0x0 + 0x1)) + (DEFINED (UsageFault_Handler)?UsageFault_Handler:0x0 + 0x1))))
                0x0000000000000000                _image_start = LOADADDR (.text)
                0x0000000000000894                _image_end = (LOADADDR (.data) + SIZEOF (.data))
                0x0000000000000894                _image_size = (_image_end - _image_start)
OUTPUT(PWM_GENUINO_ANDA.axf elf32-littlearm)

.debug_info     0x0000000000000000      0x747
 .debug_info    0x0000000000000000      0x12e ./src/PWM_GENUINO_CASI.o
 .debug_info    0x000000000000012e       0x9c ./src/Timer0.o
 .debug_info    0x00000000000001ca      0x255 ./src/cr_startup_lpc175x_6x.o
 .debug_info    0x000000000000041f       0x3f ./src/crp.o
 .debug_info    0x000000000000045e      0x22c ./src/gpio.o
 .debug_info    0x000000000000068a       0xbd ./src/mainPWM.o

.debug_abbrev   0x0000000000000000      0x3c2
 .debug_abbrev  0x0000000000000000       0xdf ./src/PWM_GENUINO_CASI.o
 .debug_abbrev  0x00000000000000df       0x6a ./src/Timer0.o
 .debug_abbrev  0x0000000000000149      0x114 ./src/cr_startup_lpc175x_6x.o
 .debug_abbrev  0x000000000000025d       0x36 ./src/crp.o
 .debug_abbrev  0x0000000000000293       0xba ./src/gpio.o
 .debug_abbrev  0x000000000000034d       0x75 ./src/mainPWM.o

.debug_aranges  0x0000000000000000      0x170
 .debug_aranges
                0x0000000000000000       0x40 ./src/PWM_GENUINO_CASI.o
 .debug_aranges
                0x0000000000000040       0x28 ./src/Timer0.o
 .debug_aranges
                0x0000000000000068       0x80 ./src/cr_startup_lpc175x_6x.o
 .debug_aranges
                0x00000000000000e8       0x18 ./src/crp.o
 .debug_aranges
                0x0000000000000100       0x50 ./src/gpio.o
 .debug_aranges
                0x0000000000000150       0x20 ./src/mainPWM.o

.debug_ranges   0x0000000000000000      0x108
 .debug_ranges  0x0000000000000000       0x30 ./src/PWM_GENUINO_CASI.o
 .debug_ranges  0x0000000000000030       0x18 ./src/Timer0.o
 .debug_ranges  0x0000000000000048       0x70 ./src/cr_startup_lpc175x_6x.o
 .debug_ranges  0x00000000000000b8       0x40 ./src/gpio.o
 .debug_ranges  0x00000000000000f8       0x10 ./src/mainPWM.o

.debug_macro    0x0000000000000000     0x118c
 .debug_macro   0x0000000000000000       0x54 ./src/PWM_GENUINO_CASI.o
 .debug_macro   0x0000000000000054      0xa66 ./src/PWM_GENUINO_CASI.o
 .debug_macro   0x0000000000000aba       0x1c ./src/PWM_GENUINO_CASI.o
 .debug_macro   0x0000000000000ad6      0x100 ./src/PWM_GENUINO_CASI.o
 .debug_macro   0x0000000000000bd6      0x2d4 ./src/PWM_GENUINO_CASI.o
 .debug_macro   0x0000000000000eaa       0x76 ./src/PWM_GENUINO_CASI.o
 .debug_macro   0x0000000000000f20       0x9a ./src/PWM_GENUINO_CASI.o
 .debug_macro   0x0000000000000fba       0xb2 ./src/PWM_GENUINO_CASI.o
 .debug_macro   0x000000000000106c       0x3e ./src/Timer0.o
 .debug_macro   0x00000000000010aa       0x1d ./src/cr_startup_lpc175x_6x.o
 .debug_macro   0x00000000000010c7       0x1a ./src/crp.o
 .debug_macro   0x00000000000010e1       0x34 ./src/crp.o
 .debug_macro   0x0000000000001115       0x23 ./src/gpio.o
 .debug_macro   0x0000000000001138       0x54 ./src/mainPWM.o

.debug_line     0x0000000000000000      0x621
 .debug_line    0x0000000000000000      0x19f ./src/PWM_GENUINO_CASI.o
 .debug_line    0x000000000000019f       0xe8 ./src/Timer0.o
 .debug_line    0x0000000000000287       0xd2 ./src/cr_startup_lpc175x_6x.o
 .debug_line    0x0000000000000359       0xb5 ./src/crp.o
 .debug_line    0x000000000000040e      0x125 ./src/gpio.o
 .debug_line    0x0000000000000533       0xee ./src/mainPWM.o

.debug_str      0x0000000000000000     0x4364
 .debug_str     0x0000000000000000     0x3fda ./src/PWM_GENUINO_CASI.o
                                       0x4017 (size before relaxing)
 .debug_str     0x0000000000003fda       0x34 ./src/Timer0.o
                                       0x3db3 (size before relaxing)
 .debug_str     0x000000000000400e      0x1d6 ./src/cr_startup_lpc175x_6x.o
                                       0x2ecc (size before relaxing)
 .debug_str     0x00000000000041e4       0xe9 ./src/crp.o
                                       0x2dd9 (size before relaxing)
 .debug_str     0x00000000000042cd       0x75 ./src/gpio.o
                                       0x3741 (size before relaxing)
 .debug_str     0x0000000000004342       0x22 ./src/mainPWM.o
                                       0x3fb9 (size before relaxing)

.comment        0x0000000000000000       0x7f
 .comment       0x0000000000000000       0x7f ./src/PWM_GENUINO_CASI.o
                                         0x80 (size before relaxing)
 .comment       0x000000000000007f       0x80 ./src/Timer0.o
 .comment       0x000000000000007f       0x80 ./src/cr_startup_lpc175x_6x.o
 .comment       0x000000000000007f       0x80 ./src/crp.o
 .comment       0x000000000000007f       0x80 ./src/gpio.o
 .comment       0x000000000000007f       0x80 ./src/mainPWM.o
 .comment       0x000000000000007f       0x80 /usr/local/mcuxpressoide-10.3.1_2233/ide/plugins/com.nxp.mcuxpresso.tools.linux_10.3.0.201811011841/tools/bin/../lib/gcc/arm-none-eabi/7.3.1/../../../../arm-none-eabi/lib/thumb/v7-m/libcr_c.a(__weak__main.o)

.ARM.attributes
                0x0000000000000000       0x33
 .ARM.attributes
                0x0000000000000000       0x33 ./src/PWM_GENUINO_CASI.o
 .ARM.attributes
                0x0000000000000033       0x33 ./src/Timer0.o
 .ARM.attributes
                0x0000000000000066       0x33 ./src/cr_startup_lpc175x_6x.o
 .ARM.attributes
                0x0000000000000099       0x33 ./src/crp.o
 .ARM.attributes
                0x00000000000000cc       0x33 ./src/gpio.o
 .ARM.attributes
                0x00000000000000ff       0x33 ./src/mainPWM.o
 .ARM.attributes
                0x0000000000000132       0x33 /usr/local/mcuxpressoide-10.3.1_2233/ide/plugins/com.nxp.mcuxpresso.tools.linux_10.3.0.201811011841/tools/bin/../lib/gcc/arm-none-eabi/7.3.1/../../../../arm-none-eabi/lib/thumb/v7-m/libcr_c.a(__weak__main.o)

.debug_frame    0x0000000000000000      0x3c4
 .debug_frame   0x0000000000000000       0xb0 ./src/PWM_GENUINO_CASI.o
 .debug_frame   0x00000000000000b0       0x50 ./src/Timer0.o
 .debug_frame   0x0000000000000100      0x170 ./src/cr_startup_lpc175x_6x.o
 .debug_frame   0x0000000000000270      0x128 ./src/gpio.o
 .debug_frame   0x0000000000000398       0x2c ./src/mainPWM.o
